:02000000C8280E
:08000800C7288F00F8309D00AD
:1000100000009D0B08280F0808008F000A309E0082
:1000200005209E0B10280F0808008F0064309F00E9
:1000300005209F0B18280F0808008F006430A000CF
:100040000D20A00B20280F080800F3308D000000C1
:100050008D0B27280800FF309400010892008515B9
:100060008511940A0108120603192F281408FF3C71
:1000700093000800031020309C009B019A01990115
:100080009801930D920D910D900D9B0D9A0D990D68
:10009000980D9C0B4C2808001B30840059201A3006
:1000A00084005920193084005920183084005920C8
:1000B0004128033000078C008C1980003030000785
:1000C0008C008C1B800008008330B220180E0F3982
:1000D000852018080F39852020309D20190E0F39F2
:1000E000852019080F398520C030B2201A0E0F392B
:1000F000852020309D201A080F3985201B0E0F39CE
:1001000085201B080F3985200800F63E0318073E9E
:100110003A3E9D20080015208510303086000514D9
:1001200005100D20051405100D20051405100520DF
:100130002030860005140510003405208514950034
:1001400006080F3986001508F039860405140510D5
:10015000950E06080F3986001508F0398604051437
:100160000510003405208510950006080F3986001B
:100170001508F039860405140510950E06080F3988
:1001800086001508F03986040514051000340900AE
:10019000850186018316103085000F3086002730D8
:1001A000810000308B00831205158B200C30B220AB
:1001B0002830B220E2308E000130B22005202030FD
:1001C0009D2046309D2052309D2045309D2051304D
:1001D0009D2055309D2045309D204E309D20C030C3
:1001E000B22043309D2045309D204D309D2045302C
:1001F0009D2054309D2052309D2045309D20203040
:100200009D201D201D201D200130B220052015201D
:1002100020309D2020309D2020309D2020309D20AA
:1002200020309D2035309D2030309D2020309D2075
:10023000C030B2204D309D2048309D207A309D2026
:1002400020309D2020309D2020309D2020309D207A
:1002500020309D201D201D201D200130B2200520B2
:10026000152046309D20C630B22048309D207A307F
:100270009D2003309600E7309700810191019001A5
:100280008316851583122520000000000000000061
:10029000000000000000000000000000000000005E
:1002A00096080319562900000000592997080319D8
:1002B000712925209703FF301706031D6029960337
:1002C0000B1D6B290B11910A03196929000000000D
:1002D0005029900A50290000000000000000000092
:1002E00050298316851183122B203A206420980808
:1002F0000319990803199A0803199B0803198229FD
:100300008E0139298E0A0319862939290130B22034
:10031000052020309D2020309D2020309D20413020
:100320009D2052309D2052309D2045309D205430DC
:100330009D20C030B22020309D2041309D2055307E
:100340009D2054309D204F309D201D201D201D20BC
:080350001D201D200511AB2941
:02400E00F93F78
:00000001FF
